S1238000526164696F444D58204F7065726174696E672053797374656D204669726D776190
S123802072652076332E332E3020436F707972696768742028632920313939362D30312089
S1238040496E74657261637469766520546563686E6F6C6F676965732C20496E632E2041A5
S11680606C6C207269676874732072657365727665642ED2
S123C0008E03FFBDF05BBDEA26BDEAD9BDEC08CEEE20BDEC3FBDEFE18600CE03FFA700A692
S123C02000263B0926F7A700A6002632BDF0A518CE2000CE200086FFA700A1002620081857
S123C0400926F3BDF0A518CE2000CE20004FA700A600260A08180926F4BDF0A5201AB61013
S123C0600884EFB710083CCE80D6BDECD933BDED2533BDED257EBDEFBDEAEFF6100AC420D8
S123C080260486452016F6100AC44026048644200B8642F6100AC48026028643979D867EF9
S123C0A0970097039706BDEEE00EBDE9BEBDE9BE7D007B2703BDCC88B6106684202615B659
S123C0C0100884EFB71008CE80F4BDECD918CE0FA0BDF0AFB60E0B979C2707B6100884EFDC
S123C0E02005B610088A10B71008B6100284FCB71002CEEEA0BDEC3FCE8091BDECD918CE44
S123C1000BB8BDF0C7263DBDECAB18CE00FABDF0C72631CEEE20BDEC3FCE80A2BDECD91834
S123C120CE03E8BDF0C7261CCE80B4BDECD918CE03E8BDF0C7260DCE80C5BDECD918CE0312
S123C140E8BDF0C7BDE9BEBDECAB18CE00FABDF0AFCEEE20BDEC3F4F97879789978E978DF1
S123C16086FF9788978A978CB60E0226037EC1737EC62D867ECEE1D29781DF82867ECED021
S123C18042977EDF7FB6100284FCB710024F9776BDC51B863D97094F970ABDC529BD964348
S123C1A0BDCCF6BDC4FD9632810127098102270220EE7EC484DE0E9C0C27E5B61002880193
S123C1C0B71002B60E1327037EC249B6106484012762BDC3208600BDEA5C86A5BDEA5C86F3
S123C1E05ABDEA5C8600BDEA5CCE0000DF3ADC3D8A10DD3596374C9737DE16DF38C605CE1E
S123C2000035BDEA79DC0EC3000FF30E048FDC16DD1818CE0010DC1805DD182407C620BDDC
S123C220EA792003C6203A180926EBDC3A88FFC8FFBDEA71863D9709DE0EEC00DD14DE0E8E
S123C240DC0EE304DD0E7EC1A0B61064840126037EC30B8600BDEA5C86A5BDEA5C865ABDC7
S123C260EA5C8600BDEA5CCE0000DF3ADE0EFC0E061AA3002302EC00C30001B30E042A0384
S123C280CC0000DD3D8A30BDEA7196374C9737BDEA5C18DE3DDC0EC3000FF30E048FDF4452
S123C2A0188C0003252AE600E1012624E10226200808088602180918091809270CE100260C
S123C2C008084C817F26F21809BDEA71DF4420D0188C0000272C86801809271108E600E175
S123C2E0012604E10227064C810026EC4A16BDEA5CDE44A600BDEA5C085AC18024F5DF4413
S123C300209EDC3A88FFC8FFBDEA71863D9709DE0EEC00DD14DE0EDC0EE304DD0E7EC1A02C
S123C320DE0EFC0E061AA3002302EC00C30001B30E042B41DD3D8300010505054C973CCEA0
S123C3408000DF18CE0000DF16CE2C00DC0EC3000FF30E04188FD63C8D435A26FBD63F5C6F
S123C360D13C25015FD73FCEC37D3A3AEC009A16DA17DD1639CC0000DD16DD3D3980004004
S123C38000200010000800040002000100008000400020001000080004000200013718EC20
S123C3A0001AA300267A18EC021AA302267718EC041AA304267418EC061AA306267118ECEF
S123C3C0081AA308266E18EC0A1AA30A266B18EC0C1AA30C266818EC0E1AA30E266518ECBF
S123C3E0101AA310266218EC121AA312265F18EC141AA314265C18EC161AA316265918EC8F
S123C400181AA318265618EC1A1AA31A265318EC1C1AA31C265018EC1E1AA31E264D2055ED
S123C420ED0018EC02ED0218EC04ED0418EC06ED0618EC08ED0818EC0AED0A18EC0CED0C11
S123C44018EC0EED0E18EC10ED1018EC12ED1218EC14ED1418EC16ED1618EC18ED1818EC4A
S123C4601AED1A18EC1CED1C18EC1EED1EDC189A16DA17DD16C6203A183ADC1804DD183327
S123C480397EC1A0DE209C1E27F7B610028801B710028600BDEA5C86A5BDEA5C865ABDEA52
S123C4A05C8600BDEA5CCE0000DF3A8620BDEA5C96284CBDEA5C96374C9737BDEA5C164FA7
S123C4C0188FDE20A600168A80BDEA5C3C08BDEA7938C6203A180926EBDC3A88FFC8FFBDDB
S123C4E0EA5C17BDEA5C863D9709DC20C304001A8328002303CC2000DD207EC1A0B61065D4
S123C50085012716F61060D741CE38003AA60026037C004086FFA70020E3395FCE38004FEF
S123C520A700085A26FA9740398600B710618603B71064BDEBB1CEC629C604BDEA79B60E98
S123C540039777BDEBE28677BDEA5C866EBDEA5C86309B77813923028B27BDEA5C860DBD99
S123C560EA5CBDEBE28677BDEA5C8664BDEA5CF60E0EBDEAA8860DBDEA5CBDEBE28677BDBF
S123C580EA5C8670BDEA5C8630BB0E0ABDEA5C860DBDEA5CBDEBE28670BDEA5C8668BDEA1E
S123C5A05CF60E16BDEAA8860DBDEA5CBDEBE28670BDEA5C8664BDEA5C8631F60E101BBD09
S123C5C0EA5C860DBDEA5CBDEBE28670BDEA5C8678BDEA5C8630F60E1527014CBDEA5C862B
S123C5E00DBDEA5CBDEBE28670BDEA5C8672BDEA5CF60E152602C60F5CBDEAA8860DBDEAAE
S123C6005C9670271BBDEBE28670BDEA5C8665BDEA5C8631F60E0F1BBDEA5C860DBDEA5C83
S123C620BDEBD2CE2000DF0E397762310D867ECEE1D29781DF82867ECED091977EDF7FB6F7
S123C640100284FCB71002863D97094F970ACE2000DF0EB60E0C81FD2708BDCB344F977AB4
S123C660200ABDCB45860ABB0E03977ABDCB9BBDCDE5B6102D85042715B6102E8520270E3A
S123C680F6102F84042607860ABB0E03977A9632810127098102270220D57EC8C8DE0E9C8E
S123C6A0492719A61084F081102605BDC7152003BDC85B7F000B863D970920B3B60E0C815A
S123C6C0FF27AC81FD27A8960B810626A27F000B7D000926077D0E0C2602202018DE1427DA
S123C6E01BCE0201DF78BDCB27CE2C00A600BDCAAC08180926F6BDCA7D7EC66FCE0201DFC5
S123C700784FBDCAACCE01005FBDCAFD0926FABDCA7D7EC66FBDCB55DE0EEC10840FDD1440
S123C720F30E08DD78BDCB27A612BDC9FBDE0EEC13DD16C6153A18CE2C008D2D8D2B8D2982
S123C7408D278D258D238D218D1F8D1D8D1B8D198D178D158D138D118D0FBDCA7DBDCB863B
S123C760DE0EDC0EE304DD0E39DC1605DD16256518EC00BDCAFD18EC02BDCAFD18EC04BD89
S123C780CAFD18EC06BDCAFD18EC08BDCAFD18EC0ABDCAFD18EC0CBDCAFD18EC0EBDCAFDF4
S123C7A018EC10BDCAFD18EC12BDCAFD18EC14BDCAFD18EC16BDCAFD18EC18BDCAFD18EC65
S123C7C01ABDCAFD18EC1CBDCAFD18EC1EBDCAFDC620183A39EC0018ED00BDCAFDEC021881
S123C7E0ED02BDCAFDEC0418ED04BDCAFDEC0618ED06BDCAFDEC0818ED08BDCAFDEC0A1831
S123C800ED0ABDCAFDEC0C18ED0CBDCAFDEC0E18ED0EBDCAFDEC1018ED10BDCAFDEC1218D0
S123C820ED12BDCAFDEC1418ED14BDCAFDEC1618ED16BDCAFDEC1818ED18BDCAFDEC1A1870
S123C840ED1ABDCAFDEC1C18ED1CBDCAFDEC1E18ED1EBDCAFDC6203A183A39BDCB55DE0E77
S123C860EC10840FDD14DD72F30E08DD78BDCB27A612BDC9FBDE0EC6123A18CE2C00DC7241
S123C8802F3708E6002B1808A600BDCAAC3CDE7209DF723818A70018085D27E25A20EBC490
S123C8A07F08A600BDCAAC3CDE7209DF723818A70018085D27C85A20E8BDCA7DBDCB86DE79
S123C8C00EDC0EE304DD0E39DE499C20270FBDC9974F970B9774863D97097EC66FB60E0C39
S123C8E081FF27F681FD27F2960B810626EC7F000B7D000926057D0E0C272D4F9727CC04C3
S123C90000DD78CE2C0096279128241A8A80BDCAC93CE60008A600BDCAC95A26F738C62001
S123C9203A7C002720E020B2967426CF962897274FD62758585858495849C32C008F3C1861
S123C940388620A101260EC60D183AC60A3AC600BDC98920268622A101260EC610183AC669
S123C960083AC600BDC98920128640A101260CC616183AC6103AC600BDC98996274A9727F8
S123C98026AE86FF97747EC8FB17E000A70018EB00C47F18E70039BDCB5518DE2018A60120
S123C9A0972818A602BDC9FB4F9727CC0400DD78C603183ACE2C0096279128240A8D197C66
S123C9C0002720F3BDCB86DC20C304001A8328002303CC2000DD20393C96278A80BDCAC9E8
S123C9E018E600C41FE7005C08180818A600A700BDCAC95A26F238C6203A39D65026079745
S123CA005186FF975039169051D7514A270D8114230286145FBDCA214A26FAC601BDCA214B
S123CA20393C37CE0053D652C11425015F3A5CD75233E7003839CE0053A600AB01AB02AB8E
S123CA4003AB04AB05AB06AB07AB08AB09AB0AAB0BAB0CAB0DAB0EAB0FAB10AB11AB12AB7A
S123CA601347394F5FCE0053ED00ED02ED04ED06ED08ED0AED0CED0EED10ED1239B6102D88
S123CA8085082727B6102E854027F2B6102D8A01B7102DCE001D0926FD84FEB7102DB61020
S123CAA02D84F7B7102D8A08B7102D3937F6102DC50827133CDE78270D09C680F5102E2737
S123CAC0FBB7102FDF7838333937F6102DC508272A3CDE78272409DF78C680F5102E27FB06
S123CAE0C640F5102327FB0FC6DCFE100E3AFF1018B7102F0EC640F7102338333937F6109F
S123CB002DC508271D3CDE7827BCC680F5102E27FBB7102F0927AD09DF7838C680F5102EDF
S123CB2027FB33F7102F393C4FFE0E08BDCAAC0926FA3839CC08D0B7102DF7102C5FF71090
S123CB402BBDEA1839BDE9F6CC0400F7102BF7102CB7102D39B60E0C81FD2610B6102D85B4
S123CB6004270B967A27054A977A26028DC6B610028801F6102DC504270884FD85012702BD
S123CB808A02B7100239B60E0C81FD260D8DB6183C18CE000ABDF0AF183839867ECEBA008A
S123CBA09746DF47CE2000DF494F97328601B710618603B7106418CE0064BDF0AFBDEBB1DE
S123CBC0CECC7FC604BDEA79B60E039777BDEBE28677BDEA5C866EBDEA5C86309B77813976
S123CBE023028B27BDEA5C860DBDEA5CBDEBE2CECC83C605BDEA79BDEBE28677BDEA5C861F
S123CC0073BDEA5CF60E0DBDEAA8860DBDEA5CBDEBE28677BDEA5C8670BDEA5C8630BB0EA2
S123CC200ABDEA5C860DBDEA5CBDEBE28670BDEA5C8668BDEA5CF60E16BDEAA8860DBDEA36
S123CC405CBDEBE28670BDEA5C8664BDEA5C8631F60E101BBDEA5C860DBDEA5C9670271B3D
S123CC60BDEBE28670BDEA5C8665BDEA5C8631F60E0F1BBDEA5C860DBDEA5CBDEBD2397797
S123CC8062300D706D31300DB6100884EFB71008B6100284FCB71002CEEE20BDEC3FCE945F
S123CCA037BDECD9867ECED042977EDF7F7F008786FF9788BDE9BE7D007B26F8BDF0A5B634
S123CCC01025844027F6B710257A009ABDE9BED687D1882712C10223035FD787D788CECC48
S123CCE0F03A3AEE00DF7F9D7E968B81FF26CD39E754E7CEE984B610258440260139B71065
S123CD00257A009ABDCFCC960927054A9709202D960A26178601978986FF978A970ABD965E
S123CD2043B60E1226058600B71064D69A545454C402B6100284FC1BB710022042960A2773
S123CD40368601978986FF978A4F970AB6106484012624B6100284FDB71002CE8105BDEC54
S123CD60D918CE00FABDF0AFBDEA26BDEAD9BDEAEF8E03FF7EC168B6100284FDB71002B6B8
S123CD8010668480261F8600B71064B6100284FC8A02B71002CE80F4BDECD918CE01F4BD26
S123CDA0F0AF7ECD53BDE9BED687D1882712C11125035FD787D788CECDC33A3AEE00DF7FAB
S123CDC07E007ED042D6B4D169D252D4FBD422DD01DA1ADAD5D799D84BD911DD39DF70E051
S123CDE02AE0FDD015B610258440260139B710257A009A7C000BBDCFCC960927064A97099F
S123CE007ECE8B960A260D8601978986FF978A970ABDCA63D69A545454C402B6106684802A
S123CE2027045D27015CB6100284FC1BB71002D6755A2634B60E14810E220486FF9776BDDB
S123CE40CF11BDEBB126258677BDEA5C866EBDEA5C86309B77813923028B27BDEA5C860D64
S123CE60BDEA5CBDEBD2C6F4D77520488600B71064B6100284FC8A02B71002CE80F4BDEC8A
S123CE80D918CE01F4BDF0AF7ECD53960A270B8601978986FF978A4F970AB60E0C81FD265D
S123CEA004967A2608B6100284FDB71002C6F4D7754F9776BDE9BE968E81FF271991872632
S123CEC006968D9189270FBDECABCEEE20BDEC3F86FF978E978DD687D188271686FF978C54
S123CEE0C10E25035FD787D788CECEF53A3AEE00DF7F7E007ED091D6B4D34CD5DAD422DC43
S123CF000FDD01DA1ADAD5DDF8DF70E02AE0FDD015F60E14C10E221396774CCECF363AA16A
S123CF20002309CECF453AA600977739CECF453AA10024F520F10F070F03070B0F0103057F
S123CF4007090B0D0F0000080004080C00020406080A0C0E2705865B7EECD5863C7EECD5F1
S123CF602705865D7EECD5863E7EECD59684812E25522616968B4C978B81052605CED015ED
S123CF80DF7FDE92DF94862E97919191263CDE94A600273381FF271381FE271DC610BDEC7E
S123CFA0F1860A9B919791DF94201F08DF94BDECAB86029B9197912011860A9B919791081E
S123CFC0DF9420068601397F00844F39969B2641863D979BB60E022623960A271FB61064BD
S123CFE084012718CC00A5BDEA71CC5A00BDEA71CC3000BDEA71CCFFCFBDEA71969C27097A
S123D00081FF270D7A009C2008B610088A10B710087A009B397F0084BDECABCED020DF7F22
S123D0207C00849684811E2618CED042B60E022703CED091DF7F4F97899787978886FF97D0
S123D0408A39967D850127037C0087967D850427077C008986FF978AD689D18A2712C10F0B
S123D06025035FD789D78ACED0733A3AEE00DF827E0081E1D2E1F2E2F6E360E535E564E5A8
S123D080F2E612E62FE70FE3EDE70FE724E73CE70F967D850127037C0087967D850427091B
S123D0A07C008986FF978A978C967D85022706860D978C978AD689D18A271B968C81FF273B
S123D0C00316D789C11225035FD789D78ACED0D93A3AEE00DF827E0081E1D2E25BE2D8E3F2
S123D0E015E5A5E3C3E5C8E564E5F2E612E62FE661E70FE69BE70FE724E73CE70F967D859D
S123D10001270A9684812E25064F9784394F3986FF39967D8504263B85022642967B840675
S123D1202715968F81FE220F27034C978F7F0084969027054A97904F39D68F8610C1782597
S123D140088606C1F0250286019790967B8504260920124F978F8630979086FF0C394F97B4
S123D1608F8630979086FF0D39963281022720FC0E04DD857F0084CED181DF7FCE8122DFA1
S123D18092BDD0FD265CBDD1122207251320227ED20DDC858401C30001DD857F0084202CF2
S123D1A0DC858300028401C30001DD857F0084201B969A840726147C0084BDCF6C270C96E6
S123D1C08484078101274A8106276839DC851A83000127081A8302002702203586FF978F04
S123D1E0202FDE85BC0E042724CE0E04DC85BDEFA80817BDEFA8DC851AB30E06230BCE0E0C
S123D20006BDEFA80817BDEFA87F0084397C008739CE8116BDECD9FE0E049C85BDCF54DCF1
S123D22085CE0096BDED61BDECE3FE0E049C85BDCF6039CE8116BDECD9FE0E049C85BDCF70
S123D24054CE8080C603BDECFCFE0E049C85BDCF6039963281022724FC0E06DD857F0084D9
S123D260CED265DF7F96842605CE81C2DF92BDD0FD2675BDD1122207251320227ED307DCE4
S123D280858401C30001DD857F0084202CDC858300028401C30001DD857F0084201B969A0C
S123D2A0840726147C0084BDCF6C270C96848407810127578106277539DC851A8300012753
S123D2C0081A8302002702204286FF978F203CCE82879C9226069684812E2409862D97841C
S123D2E0FC0E04DD85DF9239DE85BC0E0425E0DE85BC0E062711CE0E06DC85BDEFA80817B9
S123D300BDEFA87F0084397C008739CE81B6BDECD9FE0E069C85BDCF54DC85CE0096BDED34
S123D32061BDECE3FE0E069C85BDCF6039CE81B6BDECD9FE0E069C85BDCF54CE8080C60373
S123D340BDECFCFE0E069C85BDCF6039963281022720FC0E08DD857F0084CED364DF7FCE92
S123D36082C4DF92BDD0FD265CBDD1122207251320227ED3DDDC858401C30001DD857F00EA
S123D38084202CDC858300028401C30001DD857F0084201B969A840726147C0084BDCF6CFD
S123D3A0270C96848407810127378106275539DC851A83000127081A8302002702202286B7
S123D3C0FF978F201CDE85BC0E082711CE0E08DC85BDEFA80817BDEFA87F0084397C008730
S123D3E039CE82B8BDECD9FE0E049C85BDCF54DC85CE0096BDED61BDECE3FE0E049C85BD0B
S123D400CF6039CE82B8BDECD9FE0E049C85BDCF54CE8080C603BDECFCFE0E049C85BDCF0C
S123D4206039B60E0397857F0084CED434DF7FCE8366DF92BDD0FD264CBDD1122204250E18
S123D440201896854C840F97857F0084202796854A840F97857F0084201B969A84072614E9
S123D4607C0084BDCF6C270C96848407810127518106276B3996852706810F2702204286A3
S123D480FF978F203C9685B10E032731CE0E03BDEFA8B60E039777BDEBB18677BDEA5C86EB
S123D4A06EBDEA5C86309B77813923028B27BDEA5C860DBDEA5CBDEBD27F0084397C00874C
S123D4C039CE8358BDECD9F60E03D185BDCF5486419B85BDECD5F60E03D185BDCF6039CEF2
S123D4E08358BDECD9F60E03D185BDCF548620BDECD5F60E03D185BDCF6039B60E0E9785FA
S123D5007F0084CED50DDF7FCE846BDF92BDD0FD264CBDD1122204250C201496854C97851E
S123D5207F0084202596854A97857F0084201B969A840726147C0084BDCF6C270C96848422
S123D540078101274981062772399685270A81FE270681FF2702203686FF978F2030968568
S123D560B10E0E2725CE0E0EBDEFA8BDEBB18677BDEA5C8664BDEA5CF60E0EBDEAA8860D16
S123D580BDEA5CBDEBD27F0084397C008739CE845BBDECD9B60E0E9185BDCF54D685C1FF80
S123D5A0270A8620BDECD5BDED0C2006CE8467BDECE3B60E0E9185BDCF6039CE845BBDEC8E
S123D5C0D9B60E0E9185BDCF54CE8080C603BDECFCB60E0E9185BDCF6039B60E0D97857FF1
S123D5E00084CED5ECDF7FCE855FDF92BDD0FD264CBDD1122204250C201496854C97857F6A
S123D6000084202596854A97857F0084201B969A840726147C0084BDCF6C270C96848407B9
S123D620810127498106276D399685270A81FE270681FF2702203686FF978F20309685B1E2
S123D6400E0D2725CE0E0DBDEFA8BDEBB18677BDEA5C8673BDEA5CF60E0DBDEAA8860DBD1D
S123D660EA5CBDEBD27F0084397C008739CE854FBDECD9B60E0D9185BDCF54D685C1FF2741
S123D68005BDED0C2006CE855CBDECE3B60E0D9185BDCF6039CE854FBDECD9B60E0D918553
S123D6A0BDCF54CE8080C602BDECFCB60E0D9185BDCF6039B60E0297857F0084CED6C6DF11
S123D6C07FCE85CBDF92967D8506270B9685880197857F00842005BDD0FD2654969A8407C1
S123D6E026147C0084BDCF6C270C96848407810127058106271B39CE85B2BDECD9F60E02DF
S123D700D185BDCF54BDD74FF60E02D185BDCF6039CE85B2BDECD9F60E02D185BDCF54CEDA
S123D7208080C608BDECFCF60E02D185BDCF60399685B10E02271496852605CE86512003CC
S123D740CE860EDF92CED75CDF7F397C008739CE85B996852703CE85C27EECE37F0084CE9A
S123D760D764DF7F967D85022629850426179684812E2404862D9784969A840726067C003B
S123D78084BDCF6C399685CE0E02BDEFA88E03FF7EC157CED015DF7F39B60E1397857F00A1
S123D7A084CED7ABDF7FCE86ADDF92967D8502270B968588FF97857F008420148504270B45
S123D7C0968588FF97857F00842005BDD0FD2654969A840726147C0084BDCF6C270C968421
S123D7E08407810127058106271B39CE8694BDECD9F60E13D185BDCF54BDD83BF60E13D17B
S123D80085BDCF6039CE8694BDECD9F60E13D185BDCF54CE8080C608BDECFCF60E13D185F5
S123D820BDCF60399685B10E13270C9685CE0E13BDEFA87F0084397C00873996852706CEB3
S123D840869B7EECE3CE86A47EECE3B60E1197857F0084CED85DDF7FCE882CDF92967D8531
S123D86002270E96854A2A02860297857F008420188504270F96854C810223014F97857F46
S123D88000842005BDD0FD2654969A840726147C0084BDCF6C270C968484078101270581E3
S123D8A006271B39CE8812BDECD9F60E11D185BDCF54BDD8F7F60E11D185BDCF6039CE883C
S123D8C012BDECD9F60E11D185BDCF54CE8080C604BDECFCF60E11D185BDCF60399685B1CC
S123D8E00E11270FBD96439685CE0E11BDEFA87F0084397C00873996854A27094A270CCE85
S123D900881D7EECE3CE88227EECE3CE88277EECE3B60E1597857F0084CED923DF7FCE890B
S123D9202EDF92967D8502270E96854A2A02860397857F008420188504270F96854C81035A
S123D94023014F97857F00842005BDD0FD2654969A840726147C0084BDCF6C270C9684844A
S123D96007810127058106271B39CE8912BDECD9F60E15D185BDCF54BDD9F7F60E15D185B6
S123D980BDCF6039CE8912BDECD9F60E15D185BDCF54CE8080C603BDECFCF60E15D185BDBC
S123D9A0CF60399685B10E1527499685CE0E15BDEFA8BDEBB18670BDEA5C8678BDEA5C8663
S123D9C030F60E1527014CBDEA5C860DBDEA5CBDEBE28670BDEA5C8672BDEA5CF60E152630
S123D9E002C60F5CBDEAA8860DBDEA5CBDEBD27F0084397C00873996854A270C4A270F4AB7
S123DA002712CE891E7EECE3CE89227EECE3CE89267EECE3CE892A7EECE3B60E0A97857F40
S123DA200084CEDA2CDF7FCE89E9DF92967D8506270B9685880197857F00842005BDD0FD39
S123DA402654969A840726147C0084BDCF6C270C96848407810127058106271B39CE89D3A9
S123DA60BDECD9F60E0AD185BDCF54BDDAC8F60E0AD185BDCF6039CE89D3BDECD9F60E0A3A
S123DA80D185BDCF54CE8080C605BDECFCF60E0AD185BDCF60399685B10E0A2727CE0E0A6D
S123DAA0BDEFA8BDEBB18677BDEA5C8670BDEA5C8630BB0E0ABDEA5C860DBDEA5CBDEBD220
S123DAC07F0084397C008739CE89DD96852703CE89E37EECE3B60E0B97857F0084CEDAE74D
S123DAE0DF7FCE8A96DF92967D8502273196852714811E2714813C2714815A271481782715
S123DB00148678201286FF200E8600200A861E2006863C2002865A97857F0084203A8504CA
S123DB20273196852714811E2714813C2714815A27148178271486002012861E200E863CCB
S123DB40200A865A20068678200286FF97857F00842005BDD0FD2654969A840726147C0033
S123DB6084BDCF6C270C96848407810127058106271B39CE8A6DBDECD9F60E0BD185BDCF65
S123DB8054BDDBD7F60E0BD185BDCF6039CE8A6DBDECD9F60E0BD185BDCF54CE8080C60410
S123DBA0BDECFCF60E0BD185BDCF60399685B10E0B2720B610087D008526078A10B71008A0
S123DBC0200584EFB710089685CE0E0BBDEFA87F0084397C0087399685272E811E27248131
S123DBE03C271A815A271081782706CE8A917EECE3CE8A8C7EECE3CE8A877EECE3CE8A82FF
S123DC007EECE3CE8A7D7EECE3CE8A787EECE3B60E0C97857F0084CEDC21DF7FCE8AFEDF27
S123DC2092967D850227219685270C81FE271081FF270886FF200A86FD200686FE20028635
S123DC400097857F0084202A850427219685271481FF270C81FD270486FF200A8600200679
S123DC6086FD200286FE97857F00842005BDD0FD2654969A840726147C0084BDCF6C270C0F
S123DC8096848407810127058106271B39CE8AD9BDECD9F60E0CD185BDCF54BDDCDDF60EB8
S123DCA00CD185BDCF6039CE8AD9BDECD9F60E0CD185BDCF54CE8080C606BDECFCF60E0C91
S123DCC0D185BDCF60399685B10E0C270C9685CE0E0CBDEFA87F0084397C0087399685279B
S123DCE01481FE270A81FD2712CE8AF07EECE3CE8AE97EECE3CE8AE27EECE3CE8AF77EEC42
S123DD00E37F0084CEDD0EDF7FCE8C35DF92967D8503261F850426179684812E2404862DB8
S123DD209784969A840726067C0084BDCF6C397C008739CED015DF7F39B60E1297857F00B5
S123DD4084CEDD4BDF7FCE8CB3DF92967D8506270B968588FF97857F00842005BDD0FD2603
S123DD6054969A840726147C0084BDCF6C270C96848407810127058106271B39CE8C99BD26
S123DD80ECD9F60E12D185BDCF54BDDDEBF60E12D185BDCF6039CE8C99BDECD9F60E12D1FC
S123DDA085BDCF54CE8080C609BDECFCF60E12D185BDCF60399685B10E12272BCE0E12BD3E
S123DDC0EFA8B60E1281FF260AB61064840126037ECD53B60E1281FF2709960A27058600D4
S123DDE0B710647F0084397C008739CE8C9F96852703CE8CA97EECE3B60E1497857F0084F7
S123DE00CEDE0ADF7FCE8E33DF92967D8502271096854A81FE2602860E97857F0084201921
S123DE208504271096854C810F260286FF97857F00842005BDD0FD2654969A840726147CC1
S123DE400084BDCF6C270C96848407810127058106271B39CE8DE7BDECD9F60E14D185BDCB
S123DE60CF54BDDED4F60E14D185BDCF6039CE8DE7BDECD9F60E14D185BDCF54CE8080C6D3
S123DE8003BDECFCF60E14D185BDCF60399685B10E14273C9685CE0E14BDEFA8B60E039735
S123DEA077968581FF2622BDEBB18677BDEA5C866EBDEA5C86309B77813923028B27BDEAB4
S123DEC05C860DBDEA5CBDEBD24F97767F0084397C0087399685273E8101274081022742A9
S123DEE08103274481042746810527488106274A8107274C8108274E81092750810A275252
S123DF00810B2754810C2756810D2758810E275ACE8DF37EECE3CE8DF77EECE3CE8DFB7EC1
S123DF20ECE3CE8DFF7EECE3CE8E037EECE3CE8E077EECE3CE8E0B7EECE3CE8E0F7EECE39F
S123DF40CE8E137EECE3CE8E177EECE3CE8E1B7EECE3CE8E1F7EECE3CE8E237EECE3CE8E8D
S123DF60277EECE3CE8E2B7EECE3CE8E2F7EECE3B60E1097857F0084CEDF82DF7FCE8F0B95
S123DF80DF92967D8506270B968588FF97857F00842005BDD0FD2653969A840726147C00E2
S123DFA084BDCF6C270C96848407810127058106271A39CE8EF7BDECD9F60E10D185BDCF8F
S123DFC0548D5AF60E10D185BDCF6039CE8EF7BDECD9F60E10D185BDCF54CE8080C603BD00
S123DFE0ECFCF60E10D185BDCF60399685B10E102727CE0E10BDEFA8BDEBB18670BDEA5CDC
S123E0008664BDEA5C8631D6851BBDEA5C860DBDEA5CBDEBD27F0084397C008739CE8F03F7
S123E02096852603CE8F077EECE3967026037EE0DFB60E0F97857F0084CEE043DF7FCE8FDD
S123E040C4DF92967D8506271096854C9171230286FF97857F00842005BDD0FD2653969A28
S123E060840726147C0084BDCF6C270C96848407810127058106271A39CE8F9FBDECD9F6E4
S123E0800E0FD185BDCF548D5AF60E0FD185BDCF6039CE8F9FBDECD9F60E0FD185BDCF54ED
S123E0A0CE8080C606BDECFCF60E0FD185BDCF60399685B10E0F2727CE0E0FBDEFA8BDEB71
S123E0C0B18670BDEA5C8665BDEA5C8631D6851BBDEA5C860DBDEA5CBDEBD27F0084397CAC
S123E0E0008739CE8FA896854C270FCE8FAF4A2709CE8FB64A2703CE8FBD7EECE3B60E166C
S123E10097857F0084CEE10FDF7FCE9054DF92BDD0FD264ABDD1122204250C201496854C11
S123E12097857F0084202596854ADD857F0084201B969A840726147C0084BDCF6C270C96BC
S123E14084840781012749810627683996858100270681FF2702203886FF978F2032968589
S123E160B10E162727CE0E169685BDEFA8BDEBB18670BDEA5C8668BDEA5CF60E16BDEAA86B
S123E180860DBDEA5CBDEBD27F0084397C008739CE9048BDECD9B60E169185BDCF544FD6D6
S123E1A085CE0096BDED61BDECE3B60E169185BDCF6039CE9048BDECD9B60E169185BDCF22
S123E1C054CE8080C603BDECFCB60E169185BDCF6039865A9784CE911A7D0E022703CE910C
S123E1E02BBDECD9CEE1E9DF827A008426037C0089397D0009272A865A9784CEE252DF82DB
S123E200963281022713DC14CE0096BDED61BDECD9CE913CBDECE32039CE914ABDECD920C9
S123E2203186F09784CEE22ADF82969A84109196272097962719B60E11CE916C8101270AEB
S123E240CE917D81022703CE915BBDECD92003BDECAB7A008426037C0089397D0009274329
S123E260865A9784CEE2CFDF82963281022719CE918EBDECD9DC14CE0096BDED61BDECE3DA
S123E280CE9194BDECE32047CE919DBDECD94FD628CE0096BDED6108BDECE3CE91A3BDEC1B
S123E2A0E3202C86F09784CEE2AEDF822000969A84109196271997962712CE91ADB61066F2
S123E2C084802703CE91BEBDECD92003BDECAB7A008426037C008939CEE2EDDF82865A971C
S123E2E08496328102260BCE91CFBDECD97A008426037C008939B6106484012614CEE30C5F
S123E300DF82865A9784CE91E0BDECD97A008426037C0089397D00092642CEE357DF82869A
S123E3205A9784B60E0C271281FE271CCE921396328102261FCE9246201ACE91F19632811D
S123E340022611CE9224200CCE9202963281022603CE9235BDECD97A008426037C0089397E
S123E360865A9784CEE3B7DF82963281012706810227282047CE9257BDECD9FC0E04CE0010
S123E38096BDED61BDECE3CE925FBDECE3FC0E06CE0096BDED61BDECE3201CC602CE808024
S123E3A0BDECF14FD6285CCE0096BDED6108BDECE3CE9263BDECE37A008426067C0089BDD8
S123E3C0C51B39963281022720865A9784CE926FBDECD9FC0E08CE0096BDED61BDECE3CE67
S123E3E0E3E4DF827A008426037C008939B61064840126077C00897C008939865A9784D69C
S123E400402746D641964081012707F60E0EC1FF271ECE38003AA600272FCE9291BDECD9E8
S123E420BDED0CCE929CBDECE3CEE472DF822042CE927DBDECD94FD640CE0096BDED61BDC3
S123E440ECE3CEE460DF822017CE92A1B60E0E81FF2703CE92B2BDECD9CEE472DF82201277
S123E4607A0084260CCE3800DF42CEE492DF822021397A00842611865A9784CE92C3BDEC26
S123E480D9CEE489DF822001397A008426037C008939865A9784CE928BBDECD9DC42833803
S123E4A000DE42A6002604085C20F84FBDED0C8620BDECD5085C7A00402751A60026040855
S123E4C05C20F84FBDED0C8620BDECD5085C7A00402739A6002604085C20F84FBDED0C8646
S123E4E020BDECD5085C7A00402721A6002604085C20F84FBDED0C8620BDECD5085C7A00C1
S123E500402709DF42CEE51BDF82200FC609CE8080BDECE3CEE529DF82200E7A0084260848
S123E520CEE492DF827EE492397A008426067C0089BDC51B39865A9784CE92D4BDECD9F659
S123E5400E0EC1FF270A8620BDECD5BDED0C2006CE8467BDECE3CEE55BDF827A00842603CF
S123E5607C008939865A9784CEE59CDF829676261DCE92E2BDECD98620F60E03D17727027D
S123E580862BBDEC8A96778B41BDEC8A200ECE92F1BDECD9B60E149785BDDED47A008426FF
S123E5A0037C008939B60E0C81FD2618967A2714865A9784CE92FFBDECD9CEE5BFDF827A16
S123E5C0008426037C008939865A9784CE9310BDECD9F60E0DC1FF2705BDED0C2006CE8532
S123E5E05CBDECE3CEE5E9DF827A008426037C008939865A9784CE931F7D0E0A2703CE9332
S123E60030BDECD9CEE609DF827A008426037C008939B60E102614865A9784CE9341BDEC6D
S123E620D9CEE626DF827A008426037C0089399670272AB60E0F2B25865A9784CE9352B67F
S123E6400E0F8100270ACE936381012703CE9374BDECD9CEE658DF827A008426037C008987
S123E66039865A9784CE9385BDECD9B60E0C270D81FE271381FD270ACE939D200DCE939171
S123E6802008CE93A32003CE9397BDECE3CEE692DF827A008426037C00893986F09784CE38
S123E6A0EE60BDEC3F9687978E9689978DCEE6B4DF8220097A008426047C008939968484A5
S123E6C00F264BCE93A9BDECD9BDCA36CE93BB4A2739CE93C44A2733CE93CD4A272DCE93B1
S123E6E0D64A2727CE93DF4A2721CE93E84A271BCE93F14A2715CE93FA4A270FCE94034A9F
S123E7002709CE940C4A2703CE93B2BDECE339861E9784BDECABCEE71BDF827A00842603A0
S123E7207C008939865A9784CE9415BDECD9CEE733DF827A008426037C008939865A9784FA
S123E740CE9426BDECD9CEE74BDF827A008426037C0089397F0084CE9448DF92CEE761DFD2
S123E7607F967D850226248504261A9684812E2404862D9784969A840726097C00847F0041
S123E7808BBDCF6C39CEE78FDF7F397C0087397F0084CE947BDF92CEE79CDF7F967D850208
S123E7A026258504261A9684812E2404862D9784969A840726097C00847F008BBDCF6C395D
S123E7C0BDEEEE7C008739BDEEEA7C0087397F0084CE94BDDF92CEE7DBDF7F967D8502264E
S123E7E0248504261A9684812E2404862D9784969A840726097C00847F008BBDCF6C39CE76
S123E800E809DF7F397C0087397F0084CE94F0DF92CEEEA0BDEC3FCEE81CDF7F9684812E2D
S123E8202404862D9784969A8407260D7C00847F008BBDCF6C968427013986A09784CE95CF
S123E84043BDECD9CEEE20BDEC3FCEE84FDF7F7A00842602200FD68456C410B6100884EFAE
S123E8601BB710083986A09784CE9554BDECD9CEE874DF7F7A008426022012D684595959B2
S123E88059C401B6100284FE1BB710023986A09784CE9565BDECD9CEE89CDF7F7A00842690
S123E8A0022013D6845959595959C402B6100284FD1BB71002397F0084CE9576BDECD9CEB0
S123E8C0E8C4DF7F967D8506260B8501260139CEE8D7DF7F3920427F0084CE9587BDECD980
S123E8E0CEE8E5DF7F967D8505260B8502260139CEE8F8DF7F3920217F0084CE9598BDEC39
S123E900D9CEE906DF7F967D8503260B8504260139CEE931DF7F39200086A09784CE95A95E
S123E920BDECD9CEE928DF7F7A008426037EE8B63986A09784CE95BABDECD9CEE940DF7F63
S123E9407A0084260220013986A09784CE95CBBDECD9CE0069C604BDECFCCEE95FDF7F7AAE
S123E9600084260220013986A09784CE95D8BDECD9969DBDECD5CEE97BDF7F7A0084260327
S123E9807C0087397F0084CE95E8DF92CEE991DF7F967D850226238504261A9684812E2439
S123E9A004862D9784969A840726097C00847F008BBDCF6C3986FF978B397C008739967B2F
S123E9C0977CB6100A438407977B987C947B977D7D007B271E4F978B969C2608B60E0B2735
S123E9E0037F007DB60E0B979C2708B6100884EFB710087EF0A5969D8142270E863EB7100A
S123EA0009B6100884DFB7100839863CB71009B6100884DFB7100839B610088A20B710089E
S123EA20863EB7100939B6105C843FB7105CB6105D8AC0B7105DB6105F847FB7105F868315
S123EA40B710638600B71064CC0030B71061F710608603B710638601B7106239373CF61037
S123EA6065C42027F9B7106016DE3A3ADF3A383339368DE8178DE5323936A6008DDE085A95
S123EA8026F83239363CE600178DD15D2708A6018DCA085A26F838323936A6008DBE81FFC8
S123EAA02705085A26D4323936373C1754545454CEEAC93A16A600BDEA5CC40FCEED513ABC
S123EAC0A600BDEA5C3833323930313233343536373839616263646566B610088A08B7102A
S123EAE008B610098A08B710098603B7106439CE000018CE001FC605BDF0A5B6102584404D
S123EB002707B7102518092720B61065840127E8B6106081762603CE00688C000027D9C1E7
S123EB200027D5A700085A26CF86FFDE698C332E2608DE6B8C343026014F97704FDE6B8C16
S123EB403739250986018C3830250286029771CE0068A60081762606A602812E270CCE008A
S123EB6068CC2D2DED00ED02A70418CE0032BDF0AF8D3ECEEBA8C603BDEA79BDEBE2CEEBB0
S123EB80ABC606BDEA7918CE0064BDF0AF8683B71063CC0004B71061F710608603B71063EF
S123EBA0860DBDEA5C8D2B396D300D73643030390DB6106197678600B710618607B710621A
S123EBC0B61065844027F9B6100884F7B710087EEBE28D0E9667B71061B610088A08B710D8
S123EBE00839CE0007BDF0A5B6102584402706B71025092710B61065840127E9B61060813A
S123EC003E26E24F3986FF398600B71001B6100284E3B71002B610038A1CB7100318CE00FF
S123EC200FBDF0AF86388D4318CE0005BDF0AF860C8D3886068D3486018D307F009E3986CC
S123EC40408D28C640A6008D41085A26F839377F1001F61002C4FBCA08F71002CA10F7103E
S123EC6002B61000C4EFF7100233398D5037B71000C6FFF71001F61002C4F3F71002CA1056
S123EC80F71002C4EFF7100233398D3137B71000C6FFF71001F61002CA04C4F7F71002CA52
S123ECA010F71002C4EFF7100233393686018DBB7F009E32397F009E4F8A8020AE368D8EED
S123ECC04D2BFB3239367C009E969E8109260486C08D9832398DEE20B13686808D8D7F0023
S123ECE09E200136A60027078DDB8D9E0820F53239368680BDEC6B7F009E2001365D270ADA
S123ED00A6008DC18D845A0820F3323936378641C10A2505C00A4C20F7BDECD5178B30BDA7
S123ED20ECD533323936373C969E8110221F1754545454CEED513A16A6008D89BDEC8AC44B
S123ED400FCEED513AA600BDECC5BDEC8A38333239303132333435363738394142434445E1
S123ED60466F0304368630A700A701A70224026C02320424068602AB02A702542406860415
S123ED80AB02A7025424068608AB02A7025424086C018606AB02A70254240C8603AB01A788
S123EDA0018602AB02A70254240C8606AB01A7018604AB02A70254240E6C008602AB01A75F
S123EDC0018608AB02A7025424128602AB00A7008605AB01A7018606AB02A70254240DCCD4
S123EDE00501E300ED008602AB02A702A602813A2D08800AA7026C0120F4A601813A2D0878
S123EE00800AA7016C0020F45FA600813026108620A7005CA601813026058620A7015C3941
S123EE2000000D13110F010E00001619111E101000000D13110F010100001111130D010E6E
S123EE4000001F0E040000000000040E1F00000000041E1F1E04000000000000000C0408D1
S123EE6000000D13110F010E00001619111E101000000D13110F010100001111130D010E2E
S123EE800000001B000000001818181B181818001B1B1B1B1B1B1B0000041E1F1E04000088
S123EEA01E09090E141211000000060911130D0003010D1312120F000002000604040E0024
S123EEC00000060911120C001E1F1B1B1B1F1E00111B1F1F1B1B1B001B1B1F0E1F1B1B00B2
S123EEE0FC0E001A835234260139C60120015FB6100884EFB71008CE80E3BDECD918CE038E
S123EF00E8BDF0AFCE0E0217BDEFA8CE0E038600BDEFA8CE0E04CC0001BDEFA80817BDEFDB
S123EF20A8CE0E06CC02008D7F08178D7BCE0E08CC00018D7308178D6FCE0E0A86018D6814
S123EF40CE0E0B86FF8D61CE0E0C86FF8D5ACE0E0D86AB8D53CE0E0E86FF8D4CCE0E0F864C
S123EF60FF8D45CE0E1086FF8D3ECE0E1186008D37CE0E1286FF8D30CE0E1386FF8D29CE21
S123EF800E1486FF8D22CE0E1586008D1BCE0E1686698D14CE0E00CC52348D0C08178D08FB
S123EFA018CE03E8BDF0AF3937E6001127188D18C602F7103BA700C603F7103B18CE000A29
S123EFC0BDF0AF7F103B333937C616F7103BE700C617F7103B3318CE000ABDF0AF7F103BF7
S123EFE039CEF017860BB1103F261FCEF0288626B1103C2615CEF0398601B1103D260BCEE4
S123F000F04A8610B11035260139B6100884EFB71008BDECD920FE42616420434F4E464980
S123F020472076616C75650042616420485052494F2076616C7565200042616420494E493B
S123F040542076616C7565202000426164204250524F542076616C756520008610B710353E
S123F0608618B71008863CB710098602B710028603B71003860BB7103F860EB71039860038
S123F080B710388626B7103C860DB7105D8620B7105E8603B7105F8644B7105CB610268A2A
S123F0A003B7102639CC55AAB7103AF7103A3936373C183CCE02950926FD018DE818092692
S123F0C0F318383833323936373C183CCE02950926FD8DD1BDE9BE967D2604180926ED7DD5
S123F0E0007D18383833323900010102010202030102020302030304010202030203030435
S123F100020303040304040501020203020303040203030403040405020303040304040583
S123F12003040405040505060102020302030304020303040304040502030304030404055B
S123F140030404050405050602030304030404050304040504050506030404050405050623
S123F160040505060506060701020203020303040203030403040405020303040304040513
S123F1800304040504050506020303040304040503040405040505060304040504050506E3
S123F1A00405050605060607020303040304040503040405040505060304040504050506BB
S123F1C0040505060506060703040405040505060405050605060607040505060506060783
S10BF1E00506060706070708EF
S1238080202020202020202020202020202020200008090A0B0C0D0E0F202076332E332E08
S12380A03000436F090B7269086874202739362D303120002020496E74657261637469764A
S12380C06520202000546563686E6F6C6F0869657320496E630052414D20546573743A201E
S12380E0202000526573657474696E0820454550524F4D005246204D6F64756C6520457209
S1238100726F7220005475726E696E0820526164696F204F6E0046697273742044696D3AF8
S12381202000FF5365747320746865206E756D626572206F662074686520666972737420B5
S123814020202064696D6D657220746861742077696C6C6265207472616E736D6974746562
S123816064202066726F6D2074686520696E0975742020444D58207369086E616C2E202083
S1238180202020FF546869732073657474696E08206973206F6E6C0B207573656420666FEF
S12381A072202020444D582009726F746F636F6C2E202020FF004C6173742044696D3A2020
S12381C02000FF5365747320746865206E756D626572206F6620746865206C617374202069
S12381E020202064696D6D657220746861742077696C6C6265207472616E736D69747465C2
S123820064202066726F6D2074686520696E0975742020444D58207369086E616C2E2020E2
S1238220202020FF43616E6E6F74206265206C6F776572207468616E2074686520666972BB
S12382407374202064696D6D6572206E756D6265722E2020FF546869732073657474696E10
S123826008206973206F6E6C0B207573656420666F72202020444D582009726F746F636F42
S12382806C2E202020FF0043616E6E6F74206265206C6F776572207468616E20274669721B
S12382A073742044696D2773657474696E082E2020202020202020005374617274204469CA
S12382C06D3A2000FF5365747320746865206E756D626572206F66207468652073746172FB
S12382E074696E082064696D6D657220746861742077696C6C6265206F7574097574206629
S1238300726F6D202074686520726563656976656420444D587369086E616C2E202020204D
S12383202020202020FF546869732073657474696E08206973206F6E6C0B207573656420E2
S1238340666F72202020444D582009726F746F636F6C2E202020FF004E6574776F726B20C7
S123836049443A202000FF536574732074686520202020202020204E6574776F726B2049A0
S123838044207573656420746F207472616E736D697420646174616F6E6C0B20746F206D91
S12383A061746368696E087265636569766572732E202020202020FF526563656976657250
S12383C073206D7573742020757365207468652073616D65202020204E6574776F726B20FF
S12383E04944206173202020746865207472616E736D69747465722EFF526563656976658A
S12384007273207573696E08206120646966666572656E7420202020204E6574776F726BAA
S12384202049442077696C6C206E6F742072656365697665206461746166726F6D207468D5
S12384406973202020202020207472616E736D69747465722E20202020FF00547820746F23
S123846020526376723A00416C6C005365747320746865204944206F662020746865207233
S12384806563656976657220202020746861742077696C6C20202020202020726563656904
S12384A0766520646174612020202066726F6D2074686973202020202020207472616E730F
S12384C06D69747465722E20202020FF43686F6F73696E082027416C6C27202077696C6CFC
S12384E020656E61626C6520616C6C20726563656976657273206F6E20202020746869737B
S1238500206E6574776F726B2E202020FF5573696E0820612073696E086C652020726563BB
S123852065697665722049442077696C6C696E6372656173652072616E08652020616E640C
S123854020096572666F726D616E63652EFF0052656365697665722049443A002D2D00FF2A
S1238560536574732074686520756E690A75652052656365697665722049442075736564D4
S1238580746F206964656E7469660B2074686973726563656976657220746F207468652035
S12385A07472616E736D69747465722E20202020FF00526164696F3A005472616E736D6946
S12385C07400526563656976652000FF53657473207468697320726164696F20756E6974BB
S12385E020746F2065697468657220207472616E736D6974206F72202020202072656365E1
S123860069766520646174612E202020FF004368616E086520726164696F20746F207265BB
S12386206365697665723F20202020202020FF5072657373200D20666F7220596573206127
S12386406E64200C20666F72204E6F2E202020FF004368616E086520726164696F20746F2E
S1238660207472616E736D69747465723F20202020FF5072657373200D20666F72205965DC
S12386807320616E64200C20666F72204E6F2E202020FF0053656E643A200046756C6C207C
S12386A0444D58004368616E0865732000FF53657473207468652077610B2020202064610C
S12386C0746120697320656E636F6465642061732069742069732073656E7420746F726532
S12386E0636569766572732E202020202020FF2746756C6C20444D58272073656E647374FD
S1238700686520656E7469726520444D5820207369086E616C2E2054686973202020206DA6
S12387206F64652008756172616E74656573207468617420656163682075096461746577D8
S1238740696C6C2061727269766520696E202069747320656E74697265740B2E202020FFF1
S1238760274368616E086573272073656E6473206F6E6C0B20746865206368616E086573A1
S12387806265747765656E20750964617465732E54686973206D6F64652069732020202035
S12387A06661737465722062757420686173202074686520706F73736962696C69740B205B
S12387C06F662070726F647563696E082020202075096461746573207769746820202020C9
S12387E064696D6D6572206C6576656C7320202066726F6D2009726576696F7573202020A2
S1238800750964617465732E2020202020202020FF0050726F746F636F6C3A2000417574C2
S12388206F00444D5820004C57522000FF5365747320746865206461746120202009726FA4
S1238840746F636F6C207573656420620B526164696F444D582E20202020202020FF274445
S12388604D582720697320666F72202020207374616E6461726420444D582D3531326C6951
S1238880086874696E0820636F6E74726F6CFF274C57522720697320666F72202020204883
S12388A069086820456E6420530B7374656D7309726F097269657461720B20202020206372
S12388C06F6E74726F6C6C6572732E20202020FF274175746F2720616C6C6F77732020209A
S12388E0616E0B20737509096F7274656420202009726F746F636F6C20746F2062652020CD
S1238900757365642E2020202020202020202020FF00526564756E64616E63793A004F6619
S12389206600203278002033780020347800FF536574732074686520616D6F756E74206F2A
S12389406620726564756E64616E630B20696E746865207472616E736D6974746564206443
S1238960617461200961636B6574732E202020FF4120327820726564756E64616E630B2082
S12389806C6576656C2073656E647320656163687509646174652074776963652E202020E7
S12389A0FF4120686908686572206C6576656C20206D610B20646563726561736520746892
S12389C06575096461746520726174652E20202020FF00547820506F7765723A00203130E5
S12389E06D57003130306D5700FF536574732074686520616E74656E6E61096F7765722070
S1238A007573656420746F2020207472616E736D6974206461746120746F6F7468657220CD
S1238A20756E6974732E20202020FF466F72207665720B20636C6F7365202072616E08658F
S1238A400F20746865203130206D5773657474696E082073686F756C6420206265207573E0
S1238A6065642E2020202020202020FF004261636B6C690868743A004F66662000203330DA
S1238A807300203630730020393073003132307300204F6E2000FF53657473207468652048
S1238AA074696D65722020666F72206175746F6D617469632020204C4344206261636B6CD3
S1238AC06908687420202073687574206F66662E20202020202020FF0044726F09205278A1
S1238AE03A00426C61636B2000486F6C6420200053746F092020005969656C642000FF538C
S1238B006574732074686520616374696F6E20746861742077696C6C206F63637572206998
S1238B206620746865207265636569766572206C6F6F73657320636F6E746163742020777D
S1238B406974682074686520202020202020207472616E736D69747465722E20202020FF01
S1238B6027426C61636B2720086F657320746F206120626C61636B207363656E652E20201A
S1238B80FF27486F6C642720686F6C6473207468656C617374207363656E652E20202020D2
S1238BA020FF2753746F0927206361757365732020207468652072656365697665722074B7
S1238BC06F2073746F092073656E64696E0820202020646174612E20202020202020202092
S1238BE02020FF275969656C642720616C6C6F7773202074686973207265636569766572CE
S1238C0020746F6175746F6D61746963616C6C0B2020206261636B2D750920616E6F74686C
S1238C20657220736F75726365206F6620646174612E20FF005309656369616C204F097466
S1238C40696F6E733FFEFF5072657373200D20746F2075736520207309656369616C206D2A
S1238C60656E7573206F7209726573732053656C65637420746F2072657475726E20746F28
S1238C80207374617475736D6F64652E2020202020202020202020FF0052463A2020004187
S1238CA075746F204F6E202000416C77610B73204F6E0053656C65637473206966207261A6
S1238CC064696F636F6E746163742069732020202020206D61696E7461696E65640F2065FE
S1238CE076656E7768656E206E6F2064617461206973206265696E082073656E7420620B95
S1238D00202020746865207472616E736D69747465722EFF274175746F204F6E2720616CF3
S1238D206C6F7773746865207472616E736D697474657220746F207368757420646F776E8D
S1238D40202020207768656E207468657265206973206E6F6461746120696E0975742E20DB
S1238D6020202020FF416674657220746865202020202020207472616E736D697474657280
S1238D80206861732073687574206F66660F206974206D610B74616B6520736576657261E4
S1238DA06C202020207365636F6E647320666F722074686520726563656976657273207490
S1238DC06F2020202072652D61630A75697265207468652020726164696F207369086E6196
S1238DE06C2E202020FF004175746F205365656B3A20004F666600410E5000410E48004941
S1238E000E5000410E4400450E4800490E4C004D0E5000410E4200430E4400450E4600476E
S1238E200E4800490E4A004B0E4C004D0E4E004F0E5000FF53656C656374732069662072E9
S1238E406164696F6175746F6D61746963616C6C0B202020736561726368657320666F7251
S1238E60206120206E6574776F726B20776974682020202076616C6964206461746120627B
S1238E8065696E087265636569766564206F6E2069742E20FF43686F6F736520276F666619
S1238EA02720746F2064697361626C65207468697320202020666561747572650F206F723C
S1238EC0202020202063686F6F736520612072616E086520206F66206E6574776F726B736C
S1238EE0207468617477696C6C206265207365617263686564FF0044697665727369740B4B
S1238F003A20004F6666004F6E2000FF416C6C6F777320526164696F444D5820746F206F00
S1238F20096572617465207769746820612064697665727369740B2D740B0965616E74655F
S1238F406E6E612E2020202020202020FF446F206E6F74207573652074686973206F09742E
S1238F60696F6E207768656E20612020207374616E6461726420616E74656E6E61697320A2
S1238F80636F6E6E656374656420746F20526164696F444D582E20202020202020FF0043CF
S1238FA068205365743A2000476C6F62616C004672616E636500530961696E20004A610997
S1238FC0616E2000FF4C696D697473207468652052462020206368616E6E656C207365746F
S1238FE020666F7220757361086520696E207309656369616C6C6F636174696F6E732E2085
S12390002020202020FF466F72206F0965726174696F6E202020616E0B7768657265206522
S12390206C73650F20207573652074686520476C6F62616C202073657474696E082E20202D
S1239040202020202020FF00486F09204C656E0874683A00FF5468697320096172616D656A
S12390607465722020636F6E74726F6C73207468652020202073096565642061742077686E
S123908069636820206672650A75656E630B20686F707320206F636375722E202020202057
S12390A02020202020FF546865207472616E736D697474657220616E64207265636569761E
S12390C06572202020206D7573742062652073657420746F20207468652073616D65207639
S12390E0616C75652E20FF436F6E7461637420666163746F720B20666F72206D6F726520A8
S1239100696E666F2E2020FF44656661756C74203D20313035202020FF00526164696F3AD2
S123912020205472616E736D697400526164696F3A20202052656365697665002044696D13
S12391406D657220496E097574004C690868747761766520496E0975742000204E6F204488
S123916061746120496E09757420200020204E6F20444D5820496E09757420200020204E0F
S12391806F204C575220496E0975742020005265637620002044696D6D6572730052656383
S12391A0762000204669787475726573004E6F205369086E616C20446574656374004E6F89
S12391C020446174612046726F6D2054782000204C6908687477617665204461746120000B
S12391E02020526164696F206973204F666620200053656E64696E0820426C61636B6F757B
S12392007400486F6C64696E082044696D6D6572732000204F75740975742053746F0909AD
S12392206564200053656E64696E08205374616E64620B2000486F6C64696E082046697884
S1239240747572657300204F75740975742053746F09096564200054782044696D3A0020DC
S12392600E200020466978747572657320200053746172742044696D6D65723A0052656322
S12392806569766572204944733A004944733A20002052656365697665722000206973206A
S12392A00020204E6F2052656365697665727320200020205265636569766572206E6F74BF
S12392C02020002020202044657465637465642020202000547820746F20526376723A2042
S12392E020004E6574776F726B2049443A202020004E6574776F726B205365656B3A00202D
S1239300496E097574205061737374687275200052656365697665722049443A2020005456
S12393207820506F7765723A20203130206D5700547820506F7765723A20313030206D57FD
S12393400044697665727369740B20416E743A4F6E004368616E205365743A204672616ED3
S12393606365004368616E205365743A2020530961696E004368616E205365743A20204AC3
S12393806109616E0044726F092052783A20202000426C61636B0020486F6C640020537473
S12393A06F09005969656C64005369086E616C3A20002030200C0C0C0C0C002031200D0CAB
S12393C00C0C0C002032200E0C0C0C0C002033200E0D0C0C0C002034200E0E0C0C0C00202F
S12393E035200E0E0D0C0C002036200E0E0E0C0C002037200E0E0E0D0C002038200E0E0EBF
S12394000E0C002039200E0E0E0E0D003130200E0E0E0E0E0050726573732053656C656390
S12394207420746F20006368616E08652073657474696E08732E00427574746F6E73200912
S1239440726573736564200052657365742073657474696E08733F20FF5072657373200D95
S123946020666F722059657320616E64200C20666F72204E6F2E202020FF005072657373D3
S1239480200D20746F20736574750961732061207472616E736D6974746572616E64200C1D
S12394A020746F2073657475702020617320612072656365697665722E2020FF00537461B5
S12394C072742073656C6620746573743FFF5072657373200D20666F722059657320616ED9
S12394E064200C20666F72204E6F2E202020FF00FFDBDBDBDBDBDBDBDBDBDBDBDBDBDBDB33
S1239500DB313233343536373839303132333435364142434445464748494A4B4C4D4E4FF2
S1239520506162636465666768696A6B6C6D6E6F702020202008090A0B0C0D0E0F20202013
S123954020FF004261636B6C69086874206F6E2F6F666600477265656E20737461747573A2
S1239560204C45440052656420737461747573204C45442020005072657373203C53656C51
S12395806563743E2020005072657373203C446F776E3E20202020005072657373203C5590
S12395A0703E20202020202000426164206B6579207072657373656420004669726D77612D
S12395C072653A2020332E332E300052462056657273696F6E3A20005043422052657669C1
S12395E073696F6E3A20200045786974207365747570206D6F64653FFF5072657373200D0C
S123960020666F722059657320616E64200C20666F72204E6F2E202020FF00B61065851E70
S12396202606F610607E0046B610603BFC102E850E26037E0000850C26065D26037E000337
S12396407E0006B6102D84DFB7102DCEB700DF01DF04DF074F9732BDE9F6CC2400F7102B34
S1239660F7102CB7102D39B6102D84DFB7102DCEB800DF01CEB827DF04CEB899DF07CE2053
S123968000DF0CDF0ECEFFFFDF12CE2000CC0C00ED02CC0400ED04CE2400CC0800ED02CC3A
S12396A00400ED04CE2800CC0400ED02CCF800ED04BDE9F6CC2400F7102BF7102CB7102D62
S12396C039B6102D84DFB7102DCEB900DF01CEB983DF04DF07CE2000DF1EDF20BDE9F6CC77
S10F96E02400F7102BF7102CB7102D39C4
S123B700CE0204DF33CEB715DF01CEB71DDF04CEB700DF073BDE33092721DF333BDE3309D1
S123B7202719DF33C629D7023BDE3309270DDF335D2608C601D732BD96673BCE0482DF339A
S123B740CEB74BDF01CEB7A0DF043BDE33092750DF33C1802604C65BD7023BC1202708C1DE
S123B760222704C1402639C671D702CC0000DD333BC181260CDE338C000C2D24C68CD70258
S123B7803BDE33088C00162E17DF333BC1202708C1222704C1402608C602D732BD96C13BB0
S106B7A07EB7006D
S123B8003BC1002605C60FD7023BC600D7023B5D26015CDE10E71008DF108F5D26088401DF
S123B8202604860097023B86019702DC1084031A9312265EFD20002759CC2400910E274D0A
S123B840970CDD10C649D7053B86019702DC1084031A9312263CFD24002737CC2800910E68
S123B860272B970CDD10C66BD7053B86019702DC1084031A9312261AFD28002715CC2000BB
S121B880910E2709970CDD10C627D7053B960CDD103BDD12DE0CDF103BC600D7023B9C
S123B900C180260E4F9726DE1EDF2408DF22C613D7023BC180273AC58026119626811F240F
S123B9200A4C9726DE22E70008DF223BDE249626A700C47FD727C11F22124F9726585858F7
S123B9400505D31EDD24C30001DD223BC61FD7263BDE249626A7004F972696279728DC1EE5
S123B960C304001A8328002303CC20001A9320270ADD1EDD24C30001DD223BDE1EDF240826
S10BB980DF223BC600D7023BA5
S123BA00C1002604C609D7483BC1A52605C61BD7483BC1002704C600D7483BC15A2605C62A
S123BA202DD7483BC10026EEC609D7483BC10026E5DE49DF4BC63AD7483BDE4B4FDD3AC1B6
S123BA4020260BE70008DF4BCEBD00DF473BE71008DF4BC4FCC1102706C130270820B7CEE0
S10EBA60BB00DF473BCEBC00DF473BD0
S123BB00DE4BE71008DF4BDE3A3ADF3AC601D132272DD732DE49DF0ECE2000CC0C00ED0274
S123BB20CC0400ED04CE2400CC0800ED02CC0400ED04CE2800CC0400ED02CCF800ED04C69A
S123BB4044D7483BDE4BE71008DF4BDE3A3ADF3AC655D7483BDE4BE71008DF4BDE3A3ADF8E
S123BB603ACEF0E83AA600974FC66ED7483BDE4BE71008DF4BDE3A3ADF3ACEF0E83AA6004A
S123BB809B4F270B5F040404DD4DC694D7483BC6B5D7483B2719DE3A3ADF3AC10126015F74
S123BBA0DE4BE71008DF4BDE4D0927E3DF4D3BCEBA09DF473BC8FFDE4BE710C6C0D7483BD1
S123BBC0C8FFDE4BE711A6101A933A2620DE49EC10840326035D270BDC49E3041A930E2746
S119BBE002DD49B60E0D81FF2703BDEA5CCEBA00CEBA00DF473B34
S123BC00963B8403DE4BE71008DF4BDE3A3ADF3ADD4D2738C601D132272DD732DE49DF0E47
S123BC20CE2000CC0C00ED02CC0400ED04CE2400CC0800ED02CC0400ED04CE2800CC04004E
S123BC40ED02CCF800ED04C652D7483BCEBBB5DF473BDE4BE71008DF4BDE3A3ADF3AC66642
S123BC60D7484F971D3BDE4BE71008DF4BDE3A3ADF3A5D2B1AC101235E8601971A86AF97BD
S123BC80484F5CDD1BDC4D931B2E2127182048C47F5CD71A86AF97484FDD1BDC4D931B2EF8
S123BCA00B27022032DD4D86FF971D3BDD4D3BDE3A3ADF3AC10126015FDE4BE71008DF4BF2
S120BCC0961A4A2703971A3B961D2605C666D7483BCEBBB5DF473BCEBA00DF473B67
S123BD00DE4BE70008DF4BDE3A3ADF3AD7268602913227069732DE49DF20C61FD7483BDEF1
S123BD204BE70008DF4B0909A600DE3A3ADF3A4D2705C63CD7483BC67CD7483BC580277328
S123BD40DE4BE70008DF4BDE3A3ADF3AC41F2763D74DC657D7483BDE4BE70008DF4BDE3AD0
S123BD603ADF3AD64D5A2703D74D3BD6265A2707D726C63CD7483BC67CD7483BC8FFDE4BFD
S123BD80E700C687D7483BC8FFDE4BE701A6001A933A261FDC49C304001A8328002303CCC4
S123BDA020001A93202702DD49B60E0D81FF2703BDEA5CCEBA00DF473B0F8602B710021864
S123BDC0CE0032BDF0AF8600B7100218CE0032BDF0AF20E50F8601B7100218CE0032BDF017
S123BDE0AF8600B7100218CE0032BDF0AF20E50F8602B7100218CE0064BDF0AF8601B71074
S10DBE000218CE0064BDF0AF20E587
S123BFBFCF00000000000000000000000000000000000000000000962CBDB9BDB9BDB9BDAE
S123BFDFB9BDB9BDB9BDB9BDB9BDB9BDB9BDB9BDB9BDB9961BBDB9BDB9BDEFC000C000C0D6
S104BFFF003D
S123FFBFCF00000000000000000000000000000000000000000000962CBDB9BDB9BDB9BD6E
S123FFDFB9BDB9BDB9BDB9BDB9BDB9BDB9BDB9BDB9BDB9961BBDB9BDB9BDEFC000C000C096
S104FFFF00FD
S9030000FC
